:020000040800F2
:1000000000800120ED290008051B0008071B0008DF
:10001000091B00080B1B00080D1B00080000000056
:100020000000000000000000000000000F1B00089E
:10003000111B000800000000131B0008151B00081E
:100040003D2A00083D2A00083D2A00083D2A0008F4
:100050003D2A00083D2A00083D2A00083D2A0008E4
:100060003D2A00083D2A00083D2A00083D2A0008D4
:100070003D2A00083D2A00083D2A00083D2A0008C4
:100080003D2A00083D2A00083D2A00080000000023
:100090000000000000000000000000003D2A0008F1
:1000A0003D2A00083D2A00083D2A00083D2A000894
:1000B0003D2A00083D2A00083D2A00083D2A000884
:1000C0003D2A00083D2A00083D2A00083D2A000874
:1000D0003D2A00083D2A00083D2A000800000000D3
:1000E0003D2A00083D2A00083D2A000800000000C3
:1000F0000000000000000000000000003D2A000891
:10010000000000003D2A00083D2A00083D2A0008A2
:1001100000000000000000000000000000000000DF
:100120003D2A00083D2A00083D2A00083D2A000813
:100130003D2A000800000000000000000000000050
:100140000000000000000000000000003D2A000840
:100150003D2A00083D2A00083D2A00083D2A0008E3
:100160003D2A00083D2A00080000000000000000B1
:10017000000000000000000000000000000000007F
:10018000000000003D2A0008000000000000000000
:040190003D2A0008FC
:1001C0000348044B834202D0034B03B118477047E6
:1001D0007000002070000020000000000548064963
:1001E0000B1AD90F01EBA301491002D0034B03B145
:1001F00018477047700000207000002000000000C9
:1002000010B5064C237843B9FFF7DAFF044B13B15E
:100210000448AFF300800123237010BD700000205C
:1002200000000000402A000808B5044B1BB1044937
:100230000448AFF30080BDE80840CFE700000000AD
:1002400074000020402A0008014B1868704700BF66
:100250000000002070B50D4E0D4D761BB61006D077
:10026000002455F8043B01349847A642F9D1094EC1
:10027000094D761B02F0E4FBB61006D0002455F8B9
:10028000043B01349847A642F9D170BDA82C000860
:10029000A82C0008AC2C0008A82C0008024B014632
:1002A000186800F059B900BF00000020024B014659
:1002B000186800F0EFB800BF00000020844641EA53
:1002C000000313F003036DD1403A41D351F8043BCE
:1002D00040F8043B51F8043B40F8043B51F8043B20
:1002E00040F8043B51F8043B40F8043B51F8043B10
:1002F00040F8043B51F8043B40F8043B51F8043B00
:1003000040F8043B51F8043B40F8043B51F8043BEF
:1003100040F8043B51F8043B40F8043B51F8043BDF
:1003200040F8043B51F8043B40F8043B51F8043BCF
:1003300040F8043B51F8043B40F8043B51F8043BBF
:1003400040F8043B51F8043B40F8043B403ABDD22E
:10035000303211D351F8043B40F8043B51F8043BD0
:1003600040F8043B51F8043B40F8043B51F8043B8F
:1003700040F8043B103AEDD20C3205D351F8043B5F
:1003800040F8043B043AF9D2043208D0D2071CBF2B
:1003900011F8013B00F8013B01D30B880380604654
:1003A000704700BF082A13D38B078DD010F00303CA
:1003B0008AD0C3F10403D21ADB071CBF11F8013B3A
:1003C00000F8013B80D331F8023B20F8023B7BE789
:1003D000043AD9D3013A11F8013B00F8013BF9D2B4
:1003E0000B7803704B7843708B788370604670474E
:1003F000830730B548D0541E002A3FD0CAB2034606
:1004000001E0013C3AD303F8012B9D07F9D1032CFD
:100410002DD9CDB245EA05250F2C45EA054536D93B
:10042000A4F1100222F00F0C03F1200EE6444FEA73
:10043000121C03F1100242E9045542E90255103240
:100440007245F8D10CF1010214F00C0F03EB02120B
:1004500004F00F0C13D0ACF1040323F003030433B6
:10046000134442F8045B9342FBD10CF003042CB11B
:10047000CAB21C4403F8012B9C42FBD130BD644638
:100480001346002CF4D1F9E703461446BFE71A4699
:10049000A446E0E7002958D030B551F8043C83B0B9
:1004A000002BA1F10404B8BFE418019000F076F924
:1004B000284A0198136833B1A3420DD9216804EB8F
:1004C000010C63452FD06360146003B0BDE8304079
:1004D00000F066B9A34210D81A465B68002BF9D128
:1004E000116802EB010C644519D02FD3636054608E
:1004F00003B0BDE8304000F053B9116802EB010CC5
:10050000A44516D022D8216804EB010C6345EDD137
:100510001D685B682944C4E900135460D5E723686B
:1005200019441160D1E71D685B682944C4E90013D0
:10053000CAE7246821445418A3421160C5D1D3E905
:1005400000432144C2E90013BFE770470C23036056
:10055000BBE700BF8C000020F8B5CD1C25F00305DB
:1005600008350C2D38BF0C25002D064623DBA9428B
:1005700021D8254F00F012F93A6822B3144603E05F
:1005800063682246FBB11C4623685B1BF8D40B2B27
:1005900015D8636894420CBF3B605360304600F04E
:1005A000FFF804F10B00231D20F00700C21A01D050
:1005B0001B1AA350F8BD0C2333600020F8BD236044
:1005C0001C442560EAE77968C9B12946304600F045
:1005D0001DF8431C0CD0C41C24F00304A04205D019
:1005E000211A304600F012F8013001D02560D5E71D
:1005F0000C233046336000F0D3F80020F8BD3046BD
:1006000000F004F87860E0E78C00002038B5074D72
:100610000022044608462A6002F0C4F9431C00D0B8
:1006200038BD2B68002BFBD0236038BD9400002020
:100630000CB410B59CB01EAB6FF00044CDE90614AD
:100640000291084953F8042B059102A901930494DF
:1006500000F086F9029B00221A701CB0BDE8104021
:1006600002B070470802FFFF0EB410B59DB06FF0E6
:1006700000411FABCDE906010491094953F8042B51
:100680000290084C0868019302A9059400F068F9EB
:10069000029B00221A701DB0BDE8104003B07047E5
:1006A000000000200802FFFF000000000000000022
:1006B000000000000000000000000000000000003A
:1006C00090F800F06DE9024520F007016FF0000C92
:1006D00010F0070491F820F040F049804FF000043A
:1006E0006FF00700D1E9002391F840F000F1080015
:1006F00082FA4CF2A4FA8CF283FA4CF3A2FA8CF34D
:100700004BBBD1E9022382FA4CF200F10800A4FAB3
:100710008CF283FA4CF3A2FA8CF3E3B9D1E9042307
:1007200082FA4CF200F10800A4FA8CF283FA4CF33E
:10073000A2FA8CF37BB9D1E9062301F1200182FAF8
:100740004CF200F10800A4FA8CF283FA4CF3A2FAFE
:100750008CF3002BC6D0002A04BF04301A4612BA0C
:10076000B2FA82F2FDE8024500EBD2007047D1E90F
:10077000002304F00305C4F100004FEAC50514F09E
:10078000040F91F840F00CFA05F562EA05021CBF6F
:1007900063EA050362464FF00004A9E7704700BF13
:1007A000704700BF2DE9F0478F689F420C461D46F9
:1007B000164638D88246888910F4906F0ED10868A2
:1007C0003D462A46314600F023FCA2682368D21B2E
:1007D0002B44A26023600020BDE8F0874B690969C3
:1007E00003EB4308236808EBD878A3EB01096B1CE3
:1007F0004FEA68084B444345424684BF9846424608
:10080000430513D511465046FFF7A6FE074608B329
:1008100021694A46FFF752FDA38923F4906343F010
:100820008003A38107E008681F46CAE7504600F02E
:100830006BFC074650B107EB0900A8EB09032761E1
:10084000C4F81480A36020602F46BAE7216950469F
:10085000FFF720FE0C23CAF80030A38943F04003C1
:100860004FF0FF30A381B7E72DE9F04F936883B0D5
:100870009146002B6ED017688D6880460C4608683C
:10088000083744E0A38913F4906F2ED0D4E90415FF
:10089000A0EB010A05EB450505EBD5750AEB060053
:1008A0006D100130A8422A4684BF05462A465B05E2
:1008B00037D511464046FFF74FFE00283BD0524641
:1008C00021690190FFF7FAFCA289019B22F4906252
:1008D00042F08002A281A5EB0A0203EB0A006561E7
:1008E000A260236120603546B2465946524600F068
:1008F0008FFBA068D9F808102368451B8E1B03EBFB
:100900000A00A5602060C9F808601EB3083757E9DF
:1009100002B6002EFAD0B542AA46B3D93546B24641
:10092000E3E7404600F0F0FB03460028D3D12169FD
:100930004046FFF7AFFD0C23C8F80030A389002222
:1009400043F040034FF0FF30A381C9E9012203B017
:10095000BDE8F08F0020C9F8040003B0BDE8F08FB7
:100960002DE9F04F92468A8915069DB0884681464A
:100970001C4603D50A69002A00F0EF800022099284
:100980009AF800307E4D039420228DF829203022E1
:100990008DF82A200126002B72D0544603E014F86B
:1009A000013F002B76D0252BF9D1B4EB0A0B74D183
:1009B0002278002A64D000234FF0FF32CDE90523CE
:1009C000049307938DF853301A93013404E0049A8A
:1009D00006FA03F313430493A246052214F8011BFD
:1009E000284600F0C5FA431B0028F0D1049BD80626
:1009F00044BF20228DF8532019079AF8001044BFF5
:100A00002B228DF853202A2954D1039A11680432DD
:100A1000002903927CDB07919AF801100AF1010A80
:100A20002E2959D0574C0322204600F0A1FA40B19C
:100A3000049B001B402404FA00F0034304930AF1D2
:100A4000010A1AF8011B50488DF82810062200F000
:100A50008FFA002862D04D4B002B52D003AA00928F
:100A60004B4B424604A94846AFF3008007467A1C28
:100A700006D0099B3B4409939AF80030002B8CD197
:100A8000B8F80C305B0654BF09984FF0FF301DB02A
:100A9000BDE8F08FB4EB0A0BF2D05B4652464146FC
:100AA0004846FFF77FFE0130EAD0099B22785B447D
:100AB00009937EE7A1F13002092AB1D8079B1AF801
:100AC000011F03EB830302EB4303A1F13002092A68
:100AD000F5D92E290793A5D19AF801102A2927D1F3
:100AE000039B9AF802101A6805920433002A0AF14F
:100AF00002000393B8BF4FF0FF338246B8BF05939F
:100B000090E7039B073323F0070308330393B0E711
:100B1000494243F00203079104937DE703AA009240
:100B20001B4B424604A9484600F0CAF807469EE718
:100B3000A1F130020023092A05930AF1010A3FF6C8
:100B400071AF1AF8011F03EB830302EB4303A1F11A
:100B50003002092AF5D9059364E74021FFF7FCFC30
:100B6000C8F80000C8F8100018B14022C8F81420D6
:100B700004E70C23C9F800304FF0FF3087E700BFCF
:100B8000642C00086C2C0008702C00080000000089
:100B9000A50700082DE9F84F92461F460A698B68A1
:100BA000DDF828909A42B8BF1A46CAF8002091F89A
:100BB00043300C46064613B10132CAF800202268C1
:100BC00091065DD5DAF800300233CAF800302268A9
:100BD00012F0060F11461ED1E168CB1A002BD8BFC8
:100BE000114618DD04F1190B4FF0000805E0E56827
:100BF000DAF80030ED1A45450CDD01235A46394636
:100C00003046C847013008F10108F0D14FF0FF30FD
:100C1000BDE8F88F216894F84330003B18BF0123EA
:100C20008A060AD5E1185A1C302081F84300224474
:100C300094F8451082F84310023304F14302394618
:100C40003046C8470130E1D0236803F00603042B87
:100C50001DD0A3682269934225DD4FF000089B1A3E
:100C600098441A34002501E045451CDA0123224648
:100C700039463046C847013005F10105F4D1C5E7D2
:100C800012F0060F12D0003B18BF0123D5E7DAF8A7
:100C90000030E1682269C91AA368934221EAE17829
:100CA000DDDC0029DDDC0020BDE8F88FE168DAF842
:100CB0000030CB1A002BD8BF114693DCABE700BF46
:100CC0002DE9F0470C4684B09046227E0C990746E9
:100CD000994604F14300002A33D0A2F15803DDB253
:100CE000202D67D8202B65D8DFE813F0DE006400E4
:100CF00064006400640064006400640064006400D4
:100D00006400A3006E0064006400640064006E0070
:100D1000640064006400640021007F00C00064007F
:100D20006400AE0064007F0064006400E500236896
:100D30001A0640F104810B6862691D1D0D601B6875
:100D40001A60002382462361CDF80090434603AA2F
:100D500021463846FFF71EFF013020D02369524656
:100D600041463846C847013019D02368E068039EE1
:100D70009B0719D5831B002B16DD04F1190A0025EA
:100D800004E0E068039E831BAB420DDD0123524665
:100D900041463846C847013005F10105F1D14FF011
:100DA000FF3004B0BDE8F087B042B8BF304604B0B1
:100DB000BDE8F087012384F84220236104F1420A50
:100DC000002384F84330BFE723681A0602D45E0686
:100DD00000F1C1800D682A6804350D601546002AAF
:100DE0006BDBDFF884C10A2610E023681D0640F1A2
:100DF0009C800B681D1D0D601D68DFF86CC16F2A9B
:100E00000CBF08260A26002384F843306268A260DB
:100E1000002A7FDB236823F004032360002D5BD1CD
:100E2000002A79D18246082E65D0A0EB0A00206105
:100E30008AE70B680122186804330B6004F1420A48
:100E400084F842002261BBE70B686268181D0860E5
:100E5000D3F800A00021504600F08AF8002800F0E6
:100E60008180A0EB0A0060602061A9E7236843F05D
:100E7000200323607822DFF8F4C084F845200A6854
:100E8000151D0D601D0643D4590641D51588DE0792
:100E900044BF43F020032360002D44D1236823F096
:100EA000200323601026AEE7582384F84530DFF88E
:100EB000B8C02368E3E72368DCE76268A2602D21FD
:100EC000002AC5F1000584F8431002DB23F0040377
:100ED0002360DFF894C00A268246B5FBF6F306FBD2
:100EE00013512A461CF801100AF8011DB2421D4692
:100EF000F3D2082E99D12368D90796D56268236961
:100F00009A4292DC30230AF8013C0AF1FF3A8CE75E
:100F10001568BCE7002DDFD19CF8003084F8423022
:100F200004F1420A7FE710266DE713F0400F0B68CB
:100F300003F104050D600CBF1D681D885DE713F00B
:100F4000400F0B68626903F104050D601B6814BF54
:100F50001A801A60F5E60A68B2F9005004320A6095
:100F60002A463CE760687FE7782C00088C2C000854
:100F700001F0FF01102A2BDB10F0070F08D010F84A
:100F8000013B013A8B422DD010F0070F42B3F6D14E
:100F9000F0B441EA012141EA014122F007047FF067
:100FA00000070023F0E80256083C85EA010586EABE
:100FB000010685FA47F5A3FA87F586FA47F6A5FAFA
:100FC00087F68EB9EED1F0BC01F0FF0102F0070206
:100FD00032B110F8013B013A83EA010313B1F8D1B1
:100FE0000020704701387047002D06BF3546033892
:100FF000073815F0010F07D1013015F4807F02BFCB
:10100000013015F4C03F0130F0BC0138704700BF1B
:1010100088420DD98B1883420AD900EB020CBAB171
:10102000624613F801CD02F801CD9942F9D170471B
:101030000F2A0ED8034602F1FF3C4AB10CF1010C15
:10104000013B8C4411F8012B03F8012F6145F9D1C4
:10105000704740EA01039B0750D1A2F1100370B51D
:1010600001F1200C23F00F0501F1100E00F1100426
:10107000AC441B095EF8105C44F8105C5EF80C5C34
:1010800044F80C5C5EF8085C44F8085C5EF8045CAC
:1010900044F8045C0EF1100EE64504F11004E9D1A9
:1010A000013312F00C0F01EB031102F00F0400EBFF
:1010B000031327D0043C24F003064FEA940C1E448B
:1010C0001C1F8E465EF8045B44F8045FB442F9D1FD
:1010D0000CF1010402F0030203EB840301EB840131
:1010E00002F1FF3C4AB10CF1010C013B8C4411F8B8
:1010F000012B03F8012F6145F9D170BD02F1FF3CCE
:1011000003469BE72246EBE7F8B51446F9B1CAB1AE
:1011100006460D4600F020F8A04202D32F4638467E
:10112000F8BD21463046FFF717FA07460028F6D0EB
:1011300022462946FFF7C2F830462946FFF7AAF9AA
:101140003846F8BD2746FFF7A5F93846F8BDBDE893
:10115000F8401146FFF700BA51F8040C0028A0F13E
:101160000400BCBF0B58C018704700BF53B94AB940
:10117000002908BF00281CBF4FF0FF314FF0FF309F
:1011800000F074B9ADF1080C6DE904CE00F006F87A
:10119000DDF804E0DDE9022304B070472DE9F047F3
:1011A000089D04468E46002B4DD18A42944669D94B
:1011B000B2FA82F252B101FA02F3C2F1200120FA2E
:1011C00001F10CFA02FC41EA030E94404FEA1C487C
:1011D000210CBEFBF8F61FFA8CF708FB16E341EA78
:1011E000034306FB07F199420AD91CEB030306F1FE
:1011F000FF3080F01F81994240F21C81023E63441F
:101200005B1AA4B2B3FBF8F008FB103344EA0344C2
:1012100000FB07F7A7420AD91CEB040400F1FF33D7
:1012200080F00A81A74240F207816444023840EA14
:101230000640E41B00261DB1D4400023C5E900434D
:101240003146BDE8F0878B4209D9002D00F0EF80D0
:101250000026C5E9000130463146BDE8F087B3FA03
:1012600083F6002E4AD18B4202D3824200F2F980EB
:10127000841A61EB030301209E46002DE0D0C5E9EE
:10128000004EDDE702B9FFDEB2FA82F2002A40F03A
:101290009280A1EB0C014FEA1C471FFA8CFE01263D
:1012A000200CB1FBF7F307FB131140EA01410EFBE1
:1012B00003F0884208D91CEB010103F1FF3802D288
:1012C000884200F2CB804346091AA4B2B1FBF7F082
:1012D00007FB101144EA01440EFB00FEA64508D9A5
:1012E0001CEB040400F1FF3102D2A64500F2BB80E2
:1012F0000846A4EB0E0440EA03409CE7C6F1200731
:10130000B34022FA07FC4CEA030C20FA07F401FA76
:1013100006F31C43F9404FEA1C4900FA06F3B1FBFF
:10132000F9F8200C1FFA8CFE09FB181140EA014164
:1013300008FB0EF0884202FA06F20BD91CEB010101
:1013400008F1FF3A80F08880884240F28580A8F159
:1013500002086144091AA4B2B1FBF9F009FB1011AB
:1013600044EA014100FB0EFE8E4508D91CEB010149
:1013700000F1FF346CD28E456AD90238614440EAEC
:101380000840A0FB0294A1EB0E01A142C846A6466C
:1013900056D353D05DB1B3EB080261EB0E0101FAF5
:1013A00007F722FA06F3F1401F43C5E90071002652
:1013B0003146BDE8F087C2F12003D8400CFA02FCA8
:1013C00021FA03F3914001434FEA1C471FFA8CFEB8
:1013D000B3FBF7F007FB10360B0C43EA064300FBA8
:1013E0000EF69E4204FA02F408D91CEB030300F146
:1013F000FF382FD29E422DD9023863449B1B89B2FD
:10140000B3FBF7F607FB163341EA034106FB0EF385
:101410008B4208D91CEB010106F1FF3816D28B4232
:1014200014D9023E6144C91A46EA004638E72E46FE
:10143000284605E70646E3E61846F8E64B45A9D2F6
:10144000B9EB020864EB0C0E0138A3E74646EAE765
:10145000204694E74046D1E7D0467BE7023B614413
:1014600032E7304609E76444023842E7704700BF7C
:1014700084B000220092154B196B41F004011963EE
:10148000196B01F00401009100990192196B41F070
:1014900080011963196B01F0800101910199029299
:1014A000196B41F001011963196B01F001010291FF
:1014B000029903921A6B42F002021A631B6B03F04B
:1014C00002030393039B04B0704700BF003802403F
:1014D00030B595B005464C221E4901A8FEF7EEFE38
:1014E000002409E0002214AB03EB840333F84C1C06
:1014F000194801F082F90134122C29DC0D2C0EDC84
:1015000045FA04F313F0010FECD0012214AB03EB06
:10151000840333F84C1C104801F06FF9EBE745FAEF
:1015200004F313F0010F09D0012214AB03EB840381
:1015300033F84C1C094801F060F9DCE7002214ABD9
:1015400003EB840333F84C1C044801F056F9D2E74E
:1015500015B030BD582A00080008024000040240BF
:1015600070B50E4615460D4C021E18BF01224FF4F1
:101570008071204601F041F9321E18BF01224FF45C
:101580000071204601F039F92A1E18BF01224FF4DC
:101590008061204601F031F970BD00BF00000240BB
:1015A00000B587B00023019302930393049305933E
:1015B00041F6F3030193012808D00223039301A904
:1015C000054801F033F807B05DF804FB01230293EE
:1015D00002230493F3E700BF0000024030B589B056
:1015E0000020FFF7DDFF6C460E4D0FCD0FC495E8D0
:1015F0000F0084E80F000024254600E00134072C8A
:101600000DDC08AB03EB840333F8201C064801F023
:10161000EDF80128F2D10123A3401D44EEE728464E
:1016200009B030BDA42A00080000024070B588B09F
:1016300006460120FFF7B4FF6C46134D0FCD0FC4D3
:1016400095E80F0084E80F00002409E0002208ABB1
:1016500003EB840333F8201C0C4801F0CEF801346E
:10166000072C0EDC46FA04F313F0010FEED0012232
:1016700008AB03EB840333F8201C044801F0BDF8E9
:10168000EDE708B070BD00BFA42A000800000240CA
:1016900038B505460C46012211461046FFF760FF9B
:1016A0002846FFF715FF2046FFF7C0FF012211462D
:1016B0000020FFF755FF002201211046FFF750FFE1
:1016C000012211460020FFF74BFF01221146104670
:1016D000FFF746FF38BD08B5AA2145F25550FFF780
:1016E000D7FF552142F6AA20FFF7D2FF802145F20D
:1016F0005550FFF7CDFFAA2145F25550FFF7C8FF1F
:10170000552142F6AA20FFF7C3FF102145F255509C
:10171000FFF7BEFF962001F027F908BD38B5044653
:101720000D46AA2145F25550FFF7B2FF552142F66A
:10173000AA20FFF7ADFFA02145F25550FFF7A8FF03
:1017400029462046FFF7A4FF38BD10B5FFF7C0FEBD
:101750000020FFF725FF012200210846FFF700FFC8
:10176000FFF73CFF0446012211461046FFF7F8FE42
:10177000204610BD38B505460C46AA2145F2555005
:10178000FFF786FF552142F6AA20FFF781FF90213F
:1017900045F25550FFF77CFF0020FFF7D6FF286089
:1017A0000120FFF7D2FF2060F02145F25550FFF7EE
:1017B0006FFF38BD30B585B00546002412E01C49E6
:1017C00001A8FEF751FF01A8FEF77AFF4FF0FF33A3
:1017D00082B201A9174800F01EFB04F00F030F2B83
:1017E00014D00134B4F5002F1FDA2046FFF7ADFF07
:1017F000C2B28DF80F20002DE1D14FF0FF3301224E
:101800000DF10F010B4800F006FBEAE70A4B1B68DD
:10181000ADF800301B0C8DF802304FF0FF33022280
:101820006946044800F0F7FADBE705B030BD00BFB9
:10183000C42A000898000020582B000870B58AB010
:101840000024059406940794089409944FF6FF73B6
:101850000593012606960225089505A9084800F07B
:10186000E5FE009401940294039404941F230093D2
:10187000019603956946034800F0D8FE0AB070BD92
:10188000000802400004024000B587B00023019325
:1018900002930393049305934FF4E06301930123B0
:1018A00002930223049301A9024800F0BFFE07B08F
:1018B0005DF804FB0000024010B50446FEF700FF8F
:1018C0004FF0FF3382B22146014800F0A4FA10BD68
:1018D0009800002010B582B00C48FFF7EDFF0024FF
:1018E0000DE04FF0FF3301220DF10701084800F031
:1018F000F8FA9DF807102046FFF710FF0134072C77
:10190000EFDD0448FFF7D8FF02B010BDCC2A000875
:1019100098000020EC2A000872B6FEE708B50A48D5
:101920000A4B03604FF4E133436000238360C360DC
:1019300003610C2242618361C36100F03CFA00B98B
:1019400008BDFFF7E9FF00BF9800002000440040F9
:1019500000B595B03022002108A8FEF749FD00230C
:101960000393049305930693079301931F4A116C05
:1019700041F080511164126C02F080520192019A80
:1019800002931B490A6822F4404242F400420A6072
:101990000A6802F440420292029A0221089101224E
:1019A0000B9210220C920E910F9310924FF4A87389
:1019B0001193042312930723139308A800F0FAFA53
:1019C00080B90F23039302210491002305934FF460
:1019D00080520692079303A800F052FD20B915B07B
:1019E0005DF804FBFFF798FFFFF796FF0038024011
:1019F0000070004070B584B000F08AFFFFF7A8FFC8
:101A0000FFF736FDFFF78AFF0020FFF7C9FDFFF75C
:101A100015FFFFF739FF02A903A8FFF7ABFE0D2062
:101A2000FEF73CFC05460D20FEF738FC0446284E28
:101A3000039A31462846FEF717FE029A31462046A1
:101A4000FEF712FE234E3046FFF736FF2248FFF71F
:101A500033FF2846FFF730FF2048FFF72DFF2046D1
:101A6000FFF72AFF3046FFF727FF05E01C48FFF786
:101A700023FF0120FFF79EFE1A48FFF71DFF1A48BB
:101A8000FFF71AFF1948FFF717FF1948FFF714FF70
:101A90004FF0FF3301220DF10701164800F021FA43
:101AA0009DF80730322B07D0332B0BD0312BDDD0F4
:101AB0001148FFF701FFDFE71048FFF7FDFEFFF7D2
:101AC0000AFED9E70E48FFF7F7FEFFF703FFD3E75B
:101AD000F82A0008042B0008342B00084C2B0008BF
:101AE000EC2B00085C2B0008A42B0008BC2B000882
:101AF000D02B000898000020382C0008002C00088B
:101B0000142C0008FEE7FEE7FEE7FEE7FEE770475D
:101B10007047704708B500F015FF08BD82B000217E
:101B200000910B4B5A6C42F480425A645A6C02F496
:101B300080420092009A01911A6C42F080521A641D
:101B40001B6C03F080530193019B02B0704700BFF0
:101B50000038024000B589B0002303930493059335
:101B6000069307930268144B9A4202D009B05DF8BD
:101B700004FB0021019103F5FA331A6C42F40032A0
:101B80001A641A6C02F400320192019A02911A6BE3
:101B900042F001021A631B6B03F001030293029BE4
:101BA0000C230393022304930723079303A90348F9
:101BB00000F03CFDDAE700BF0044004000000240B6
:101BC000026802F10C0353E8003F23F490730C32D7
:101BD00042E800310029F3D1026802F1140353E80E
:101BE000003F23F00103143242E800310029F3D111
:101BF000036B012B05D0202380F8423000230363C0
:101C00007047026802F10C0353E8003F23F0100311
:101C10000C3242E800310029F3D1ECE738B5044634
:101C20000268136923F44053C1680B43136183684E
:101C30000269134342691343C2691A430168CB68BE
:101C400023F4164323F00C031343CB60026853695B
:101C500023F4407381690B4353610368314A934213
:101C600006D002F58062934202D000F0BFFC01E092
:101C700000F0CCFCE369B3F5004F29D00021031834
:101C800049411B1841F10001C90041EA5371DB00D1
:101C9000181863684FEA83024FEA937341F1000119
:101CA000FFF764FA204DA5FB00325109642303FBC2
:101CB00011031B013233A5FB03235B0903F0F00280
:101CC00002EB011203F00F03216813448B6038BD4F
:101CD0000023021843EB0301121841F10001C9006F
:101CE00041EA5271D200101841F100016268921865
:101CF0005B41FFF73BFA0C4DA5FB00325109642311
:101D000003FB1103DB003233A5FB03235B095A00FD
:101D100002F4F87202EB011203F007032168134486
:101D20008B60D4E7001001401F85EB512DE9F04393
:101D300083B005460E4617469946DDF828802C6884
:101D4000246836EA04030CBF4FF0010C4FF0000C7E
:101D5000BC4528D1B8F1FF3FF1D000F0FFFDA0EB6A
:101D60000900404523D8B8F1000F22D02B68DA686B
:101D700012F0040FE3D0802EE1D0402EDFD01A689D
:101D800012F0080FDBD0002401941A6801925B68FE
:101D90000193019B2846FFF713FF08236B6485F826
:101DA0004040012000E0002003B0BDE8F0830320A4
:101DB000FAE70320F8E760B310B5044690F8413025
:101DC00013B3242384F841302268D36823F40053EA
:101DD000D3602046FFF722FF2268136923F4904363
:101DE00013612268536923F02A0353612268D36880
:101DF00043F40053D36000206064202384F8413012
:101E000084F84230606310BD80F84030FFF7A2FED6
:101E1000D7E7012070472DE9F04182B01E4690F8C7
:101E20004130DBB2202B56D104460D4690460029A6
:101E300055D00AB901204FE000234364212380F8E4
:101E4000413000F08BFD0746A4F82480A4F82680DA
:101E5000A368B3F5805F02D04FF0000814E0236957
:101E60002BB34FF000080FE0202384F8413003200B
:101E700032E038F8023B2268C3F308035360E28C77
:101E800092B2013A92B2E284E38C9BB293B1009693
:101E90003B46002280212046FFF748FF0028E3D17F
:101EA000002DE6D015F8012B23685A60E7E7A84615
:101EB0000025E9E700963B46002240212046FFF737
:101EC00035FF18B9202384F8413005E0202384F839
:101ED0004130032000E0022002B0BDE8F081012083
:101EE000FAE72DE9F04182B01E4690F84230DBB2AD
:101EF000202B59D104460D469046002958D00AB9E6
:101F0000012052E000234364222280F84220036330
:101F100000F024FD0746A4F82C80A4F82E80A368C6
:101F2000B3F5805F02D04FF000081CE0236913B1C5
:101F30004FF0000817E0A846002514E0202384F89D
:101F40004230032031E023685B68C3F3080328F8BC
:101F5000023B03E023685B682B700135E28D92B28F
:101F6000013A92B2E285E38D9BB2C3B100963B4643
:101F7000002220212046FFF7D9FE0028DED1002DC7
:101F8000E1D0A368B3F5805FE4D013B92369002BD7
:101F9000E0D023685B6803F07F032B70DDE720232C
:101FA00084F84230002000E0022002B0BDE8F08159
:101FB0000120FAE7002800F0E08170B582B0044605
:101FC000036813F0010F3BD09F4B9B6803F00C0399
:101FD000042B2CD09C4B9B6803F00C03082B21D0C6
:101FE0006368B3F5803F4FD0B3F5A02F52D0964B26
:101FF0001A6822F480321A601A6822F480221A6069
:102000006368002B50D000F0A9FC05468E4B1B687E
:1020100013F4003F14D100F0A1FC401B6428F5D953
:102020000320B1E1884B5B6813F4800FD8D0864B56
:102030001B6813F4003F03D06368002B00F09F81FE
:10204000236813F0020F54D07F4B9B6813F00C0FE2
:102050003ED07D4B9B6803F00C03082B33D0E36824
:10206000002B68D0794B01221A6000F077FC0546FE
:10207000754B1B6813F0020F54D100F06FFC401B2E
:102080000228F5D903207FE16F4A136843F48033B7
:102090001360B5E76C4B1A6842F480221A601A6824
:1020A00042F480321A60ABE700F058FC0546664BFC
:1020B0001B6813F4003FC3D000F050FC401B6428A1
:1020C000F5D9032060E1604B5B6813F4800FC6D143
:1020D0005D4B1B6813F0020F03D0E368012B40F047
:1020E0005081594A136823F0F803216943EAC10378
:1020F0001360236813F0080F42D063696BB3534B2E
:102100000122C3F8802E00F029FC05464E4B5B6F80
:1021100013F0020F34D100F021FC401B0228F5D946
:10212000032031E1484A136823F0F803216943EAA8
:10213000C1031360DDE7454B00221A6000F00EFC7E
:102140000546414B1B6813F0020FD2D000F006FC8D
:10215000401B0228F5D9032016E13C4B0022C3F8AE
:10216000802E00F0FBFB0546374B5B6F13F0020F30
:1021700006D000F0F3FB401B0228F5D9032003E151
:10218000236813F0040F77D02F4B1B6C13F0805F84
:1021900033D1002301932C4B1A6C42F080521A6405
:1021A0001B6C03F080530193019B0125284B1B6896
:1021B00013F4807F23D0A368012B34D0052B38D0B3
:1021C000214B1A6F22F001021A671A6F22F00402E3
:1021D0001A67A368002B3DD000F0C0FB06461A4BDF
:1021E0001B6F13F0020F46D100F0B8FB801B41F2C9
:1021F00088339842F3D90320C6E00025D6E7144A75
:10220000136843F48073136000F0A8FB0646104B7C
:102210001B6813F4807FCED100F0A0FB801B022846
:10222000F5D90320B0E0084A136F43F001031367A8
:10223000CFE7054B1A6F42F004021A671A6F42F09B
:1022400001021A67C5E700BF00380240000047429C
:102250000070004000F082FB0646524B1B6F13F0EB
:10226000020F08D000F07AFB801B41F288339842BD
:10227000F3D9032088E0EDB9A369002B00F0838037
:10228000484A926802F00C02082A51D0022B17D05B
:10229000454B00221A6600F061FB0446414B1B6867
:1022A00013F0007F42D000F059FB001B0228F5D943
:1022B000032069E03B4A136C23F080531364DBE78F
:1022C000394B00221A6600F049FB0546354B1B6866
:1022D00013F0007F06D000F041FB401B0228F5D927
:1022E000032051E0E369226A1343626A43EA8213DE
:1022F000A26A5208013A43EA0243E26A43EA0263ED
:10230000284A5360284B01221A6600F027FB044636
:10231000244B1B6813F0007F06D100F01FFB001B4D
:102320000228F5D903202FE000202DE000202BE02B
:10233000012B2BD01B4B5B6803F48001E2699142B7
:1023400026D103F03F02216A8A4223D1616A47F60F
:10235000C0721A40B2EB811F1ED103F44031A26A51
:102360005208013AB1EB024F18D103F07063E26AF0
:10237000B3EB026F14D1002006E00120704701206A
:1023800002E0012000E0002002B070BD0120FBE768
:102390000120F9E70120F7E70120F5E70120F3E745
:1023A0000120F1E7003802400000474208B5314BF8
:1023B0009B6803F00C03042B57D0082B57D12D4BEF
:1023C0005A6802F03F025B6813F4800F2AD0294B51
:1023D0005968C1F3881C4FEA4C11B1EB0C006EEB4D
:1023E0000E0E4FEA8E1343EA90638101091A63EBE4
:1023F0000E03DB0043EA5173C90011EB0C0C43F1EF
:102400000003590200234FEA4C2041EADC51FEF759
:10241000ADFE184B5B68C3F3014301335B00B0FBB7
:10242000F3F025E0134B5968C1F3881C4FEA4C11B7
:10243000B1EB0C006EEB0E0E4FEA8E1343EA906385
:102440008101091A63EB0E03DB0043EA5173C900F3
:1024500011EB0C0C43F10003990200234FEA8C208E
:1024600041EA9C51FEF782FED3E7034800E00348AF
:1024700008BD00BF0038024000127A000024F400BA
:10248000002800F09B8070B50D4604464F4B1B683A
:1024900003F007038B4208D2CBB24C4A1370136887
:1024A00003F007038B4240F08B80236813F0020F88
:1024B00017D013F0040F04D0454A936843F4E05357
:1024C0009360236813F0080F04D0414A936843F4E3
:1024D000604393603E4A936823F0F003A1680B4386
:1024E0009360236813F0010F32D06368012B21D071
:1024F0009A1E012A25D9364A126812F0020F61D0BD
:1025000033498A6822F0030213438B6000F026FAF5
:1025100006462F4B9B6803F00C036268B3EB820FF7
:1025200016D000F01BFA801B41F288339842F0D994
:10253000032042E0264A126812F4003FE0D1012055
:102540003BE0234A126812F0007FD9D1012034E029
:102550001E4B1B6803F00703AB4207D9EAB21B4BC3
:102560001A701B6803F00703AB422DD1236813F0E8
:10257000040F06D0164A936823F4E053E1680B4336
:102580009360236813F0080F07D0114A936823F46F
:102590006043216943EAC1039360FFF707FF0C4BD7
:1025A0009B68C3F303130B4AD35CD8400A4B1860F3
:1025B0000A4B186800F086F9002070BD01207047B2
:1025C0000120FAE70120F8E70120F6E7003C02408D
:1025D000003802404C2C00086C00002068000020ED
:1025E000014B1868704700BF6C00002008B5FFF76A
:1025F000F7FF044B9B68C3F38223034AD35CD840A4
:1026000008BD00BF003802405C2C000808B5FFF789
:10261000E7FF044B9B68C3F34233034AD35CD840C3
:1026200008BD00BF003802405C2C000800230F2BBF
:1026300000F2D28070B582B060E085685E0003244D
:10264000B44025EA0405CC68B4402C438460456856
:1026500025EA02054C68C4F300129A402A434260FE
:102660005AE0DC08083450F8246003F007029500B3
:102670000F22AA4026EA020E0A69AA4042EA0E0286
:1026800040F824205CE0042200E0002202FA0EF26E
:102690002A430234514D45F82420514A94686FEA88
:1026A0000C0224EA0C054E6816F4801F01D04CEA97
:1026B00004054B4CA560E46802EA04054E6816F474
:1026C000001F01D04CEA0405454CE560646802EA4D
:1026D00004054E6816F4003F01D04CEA0405404C56
:1026E0006560246822404D6815F4803F01D04CEAB3
:1026F00004023B4C226001330F2B6BD801229A401D
:102700000C6804EA020C32EA0404F4D14C6804F0C8
:102710000304013C012C90D94A6802F00302032A09
:1027200009D0C4685D000322AA4024EA02048A6832
:10273000AA402243C2604A6802F00302022A90D0F3
:1027400004684FEA430E032202FA0EF224EA02045E
:102750004A6802F0030202FA0EF2224302604A685B
:1027600012F4403FC7D0002201921E4A546C44F438
:1027700080445464526C02F480420192019A9C0895
:10278000A51C164A52F8255003F003024FEA820EA8
:102790000F2202FA0EF225EA0205134A90423FF494
:1027A00074AF02F5806290420ED002F580629042D2
:1027B0000CD002F5806290420AD002F5806290420D
:1027C0003FF461AF072261E701225FE702225DE784
:1027D00003225BE702B070BD704700BF00380140C4
:1027E000003C0140003802400000024003691942E9
:1027F00001D001207047002070470AB18161704705
:102800000904816170470000074AD36823F4E0633C
:102810001B041B0C000200F4E060034343F0BF63A1
:1028200043F40033D360704700ED00E000B5194B6E
:10283000DB68C3F30223C3F1070CBCF1040F28BF0C
:102840004FF0040C03F1040EBEF1060F18D9033B40
:102850004FF0FF3E0EFA0CFC21EA0C0199400EFAF3
:1028600003F322EA0303194300280BDB0901C9B271
:1028700000F1604000F5614080F800135DF804FB52
:102880000023E5E700F00F000901C9B2024B19541B
:10289000F4E700BF00ED00E014ED00E00138B0F116
:1028A000807F0BD24FF0E0235861054AF02182F877
:1028B00023100020986107221A6170470120704799
:1028C00000ED00E010B504460E4B18784FF47A7313
:1028D000B3FBF0F30C4A1068B0FBF3F0FFF7DEFF38
:1028E00068B90F2C01D901200AE0002221464FF0DF
:1028F000FF30FFF79BFF054B1C60002000E001202C
:1029000010BD00BF640000206C00002068000020A3
:1029100008B50B4B1A6842F400721A601A6842F448
:1029200080621A601A6842F480721A600320FFF70E
:102930006BFF0020FFF7C6FFFFF7F0F8002008BD8F
:10294000003C0240034A1168034B1B780B441360A0
:10295000704700BFE000002064000020014B1868B1
:10296000704700BFE000002038B50446FFF7F6FFCF
:102970000546B4F1FF3F02D0044B1B781C44FFF71F
:10298000EDFF401BA042FAD338BD00BF6400002019
:10299000034AD2F8883043F47003C2F88830704795
:1029A00000ED00E010B503460C4A0D490D480068E3
:1029B00040B10C4800680344521A934206D8094AB1
:1029C000136010BD0748084C0460F2E7FDF73CFCBB
:1029D0000C2303604FF0FF30F3E700BF00800120BD
:1029E00000040000E4000020E8000020DFF834D0FC
:1029F000FFF7CEFF0C480D490D4A002302E0D458E2
:102A0000C4500433C4188C42F9D30A4A0A4C002338
:102A100001E013600432A242FBD3FDF71BFCFEF77A
:102A2000E9FF7047008001200000002070000020B6
:102A3000B02C000870000020E8000020FEE7000035
:102A4000F8B500BFF8BC08BC9E467047F8B500BF9B
:082A5000F8BC08BC9E4670476B
:102A5800010000000200000004000000080000005F
:102A6800100000002000000040000000800000006E
:102A7800000100000002000000040000000800003F
:102A8800001000000020000001000000020000000B
:102A98000400000008000000100000000100000011
:102AA80002000000000800000010000010000000F4
:102AB800200000004000000080000000253032584F
:102AC8002000000057616974696E6720666F722084
:102AD80066696C6520746F20666C6173682E2E2E93
:102AE8000D0A000066696E69736865640D0A000066
:102AF800307825303258200D0A0000003D3D3D3D1C
:102B08003D3D3D3D3D3D3D3D3D3D3D3D3D3D3D3DED
:102B18003D3D3D3D3D3D3D3D3D3D3D3D3D3D3D3DDD
:102B28003D3D3D3D3D3D0D0A000000004D616E7587
:102B38006661637475726572204944203D200D0AF0
:102B480000000000446576696365204944203D2003
:102B58000D0A000048656C6C6F2077656C636F6DBB
:102B68006520746F2074686520454550524F4D208C
:102B780070726F6772616D6D65722120576861743C
:102B880020776F756C6420796F75206C696B652090
:102B9800746F20646F3F0D0A000000005B315D20F8
:102BA80044756D7020526F6D206173206368617287
:102BB8000D0A00005B325D20457261736520636811
:102BC80069700D0A000000005B335D2050726F676A
:102BD80072616D2063686970207669612055415281
:102BE800540D0A0044756D70696E6720524F4D2E62
:102BF8002E2E0D0A0000000045726173696E672071
:102C0800436869702E2E2E0D0A0000004C61756E07
:102C18006368696E672070726F6772616D6D696E47
:102C2800672073657175656E63652E2E2E0D0A001B
:102C3800496E76616C696420696E707574210D0A3D
:102C48000000000000000000000000000102030472
:102C5800060708090000000001020304232D302B99
:102C680020000000686C4C00656667454647000018
:102C780030313233343536373839414243444546AA
:102C8800000000003031323334353637383961626C
:082C98006364656600000000A2
:082CA000FCE4FF7F01000000CD
:042CA80029020008F5
:042CAC000102000819
:102CB00004000020000000000000000000000000F0
:102CC0000000000000000000000000000000000004
:102CD00000000000000000000000000000000000F4
:102CE00000000000000000000000000000000000E4
:102CF00000000000000000000000000000000000D4
:102D000000000000000000000000000000000000C3
:102D10000000000001000000100000000024F4008A
:04000005080029EDD9
:00000001FF
